:100000000C9446000C940E010C940E010C940E01FD
:100010000C940E010C940E010C940E010C940E0124
:100020000C940E010C940E010C940E010C940E0114
:100030000C940E010C940E010C940E010C940E0104
:100040000C940E010C940E010C940E010C940E01F4
:100050000C940E010C940E010C940E010C940E01E4
:100060000C940E010C940E010C940E010C940E01D4
:100070000C940E010C940E010C940E010C940E01C4
:100080000C940E010C940E010C940E0111241FBE51
:10009000CFEFD0E1DEBFCDBF0E94D3000C94500063
:0400A000F894FFCF02
:0A00A40050696E74656261617300BB
:1000AE00CF938FEF84BB85BB81BB8ABB15BA1BBABE
:1000BE00C0E2C5BB0E949600C5BB0E94960080E8B8
:1000CE0085BB0E94960015BA0E94960080EF85BBF4
:1000DE000E94960015BA0E94960080E685BB0E948B
:1000EE00960082E00E94BF000E949600CF91089574
:1000FE00CF92DF92EF926B01E82E07C0862F0E94FF
:10010E00AB008FEFC81AD80AE80AF6015E2D0E94DE
:0E011E0007016111F3CFEF90DF90CF900895AD
:10012C0086E090E00E94FC0083EC99E00197F1F7E7
:10013C0000C0000086E090E00E94F00083EC99E0A3
:0A014C000197F1F700C000000895CC
:10015600CF93C82F85BB84E090E00E94FC000E94EC
:100166009600C295C07FC5BB84E090E00E94FC006B
:080176000E949600CF9108954C
:10017E00CF93C82F85BB84E090E00E94F0000E94D0
:10018E009600C295C07FC5BB84E090E00E94F0004F
:08019E000E949600CF91089524
:1001A6000E94570087EA91E60197F1F700C0000028
:1001B6000E94E30064EA70E080E00E947F00FFCFC7
:1001C60081E00E94BF0087E893E10197F1F700C044
:0A01D600000080E80E94BF000895B9
:1001E0009BB321E030E002C0220F331F8A95E2F773
:0801F000209529232BBB089583
:1001F8009BB321E030E002C0220F331F8A95E2F75B
:06020800292B2BBB089519
:0E020E0057FD03C05BBF67910895608108959E
:04021C000C9400003E
:00000001FF
